:100000000C9494020C94D8020C94D8020C94D8024C
:100010000C94D8020C94D8020C94D8020C94D802F8
:100020000C94D8020C94D8020C94E00D0C94B20EEF
:100030000C94D8020C94D8020C94D8020C94D802D8
:100040000C94D8020C946C230C94D8020C94D80213
:100050000C94D8020C94FF1C0C94D8020C94D80277
:100060000C94D8020C94D8020C94D8020C94D802A8
:100070000C94D8020C94D8020C94D8020C94D80298
:100080000C94D8020C94D8020C94D8020C94D80288
:100090000C94D8020C94D8020C94D8020C94D80278
:1000A0000C94D8020C94D8020C94D8021F0F410F64
:1000B0002F10410F2F10860FA90F2F10FE0F1110B8
:1000C000E212E2120E130E1351137113CC14CC145E
:1000D0007C13CC1429142914BD14CC14CC14C614CC
:1000E00036143614361436143614361436143614C0
:1000F00036143614361436143614361436143614B0
:10010000471454145B1462146C14021902E30001C6
:10011000E3011900020602E30001E30106000213F5
:100120000001E00104020402E001130002290001C1
:10013000E00104020402E00129000000F4A2002210
:1001400030A135002B003171C200C10000001E003B
:10015000140004001D0001544D001F001A00160079
:100160001B00E0004C002000080007000600E20031
:100170002A002100150009001900E3004A002200AE
:1001800017000A00050000000A3029006B77000004
:100190006D7F00000B3066006C7700006E7F000002
:1001A0000C3023001C000B00110000000D30240057
:1001B00018000D001000E7004B0025000C000E0099
:1001C0003600E6002C00260012000F0037002F71C9
:1001D00028002700130033003800C3004E002D0014
:1001E0002E003471C200C10000000000FF00FE00BC
:1001F000FD00000000000000000000000000010001
:100200000000F400F900F200FB0000000000F5001F
:10021000F000F100000000000000F600FA00F3001A
:10022000FC000000000000000000000000000000D2
:1002300000000000000000000000000000002B0291
:100240002B0000005800000000009C005F005C00D4
:10025000590000000000540060005D005A00620078
:100260000000550061005E005B0063000000230297
:100270005700560067008500010026022702000093
:10028000000001000000000000000000000000006D
:100290000000000000003900E100010000003A0009
:1002A000AD00B0000000000000003B00BC00AC004E
:1002B0000000010000003C00AF00AE0000000100A3
:1002C00000003D00BB00AB000000010000003E004C
:1002D000000000000000000000003F0001000000DE
:1002E00001000000000040000100000001000000CB
:1002F000000041000000500000000000000042002B
:100300000000510000000100000043000000520006
:10031000000001000000440000004F000000010048
:100320000000450000000000000000000000A900DF
:10033000AA00A800E50001000000160345007200B5
:1003400067006F0044006F007800200045005A00ED
:10035000000016034500720067006F0044006F0044
:100360007800200045005A00000004030904090237
:100370006D00040100A0FA0904000001030101005E
:10038000092111010001223F000705810308000A2D
:1003900009040100010301020009211101000122E9
:1003A0004D000705820308000A090402000103004A
:1003B000000009211101000122360007058303080E
:1003C000000A0904030001030000000921110100D3
:1003D00001223900070584031000011201100100F9
:1003E000000008EDFE0713010001020001050109EC
:1003F00006A101050719E029E715002501950875F3
:1004000001810205081901290595057501910295DB
:10041000017503910105071900297715002501953C
:100420007875018102C005010980A10185021601CC
:100430000026B7001A01002AB70075109501810047
:10044000C0050C0901A1018503160100269C021AB2
:1004500001002A9C02751095018100C00501090266
:10046000A1010901A10005091901290515002501AE
:10047000950575018102950175038101050109301A
:1004800009311581257F9502750881060938158186
:10049000257F950175088106050C0A38021581250E
:1004A0007F950175088106C0C005010906A10105F7
:1004B0000719E029E71500250195087501810295C6
:1004C0000175088101050819012905950575019136
:1004D000029501750391010507190029FF150025F3
:1004E000FF950675088100C00000000000000000B4
:1004F000000000010204060A0F17202C3A4A5D7121
:10050000879DB3C7DAE9F5FCFFFCF5E9DAC7B39DCF
:1005100087715D4A3A2C20170F0A06040201000079
:10052000000000000000000011241FBECFEFDAE041
:10053000DEBFCDBF04B603FE24C0809101029091BE
:100540000202A0910302B09104028730904BA740B1
:10055000B04BB9F410920102109202021092030201
:100560001092040214BE84B7877F84BF88E10FB65F
:10057000F89480936000109260000FBEE0E0FFE30B
:10058000099511E0A0E0B1E0E6E6FAE402C00590CA
:100590000D92A433B107D9F712E0A4E3B1E001C092
:1005A0001D92A130B107E1F70E94240B0C94312574
:1005B0000C9400001092B9008AE08093B80008956E
:1005C00094EA9093BC009091BC0097FFFCCF90916F
:1005D000B900987F983021F0903111F081E00895B2
:1005E0008093BB0084E88093BC008091BC0087FFAF
:1005F000FCCF8091B900887F883111F0803471F789
:1006000080E0089584E98093BC008091BC0084FD63
:10061000FCCF08958093BB0084E88093BC00809158
:10062000BC0087FFFCCF9091B900987F81E09832A1
:1006300009F480E0089584E88093BC008091BC00B8
:1006400087FFFCCF8091BB0008958091010181114B
:1006500015C080E40E94E0028093010181110CC06A
:1006600082E10E940A0380930101811105C08FEF8E
:100670000E940A03809301010E94020384B1807FDB
:1006800084B985B1807F85B98AB1837F8AB98BB1FE
:10069000837F8BB93E98469808950E94E00480932A
:1006A00001010E94250380B38C7080BB81B3836FEE
:1006B00081BBA5E3B1E0E3E4F1E08EE08E0F11929F
:1006C0001D928E13FCCF0C94CA04BF92CF92DF927E
:1006D000EF92FF920F931F93CF93DF9380910101CD
:1006E000882379F0809134018F5F809334018111E8
:1006F00008C00E94E00480930101811102C00E94A1
:10070000720405E311E0C0E0D0E0DD24D39482E080
:10071000C82EEE24E394F12CC730D10500F580916A
:100720000101811164C080E40E94E0028093010114
:10073000811112C082E10E940A038093010181119C
:100740000BC0C7010C2E01C0880F0A94EAF78095F0
:100750000E940A03809301010E94020348C0CA302C
:10076000A1F028F4C83059F0C93061F005C0CC3090
:1007700089F070F0CD3089F0209A289810C0219A25
:1007800029980DC0229A2A980AC0239A2B9807C04C
:10079000529A01C0539A5B9802C03E9A469890EADA
:1007A0009A95F1F79FB1799902C082E001C080E08B
:1007B00091709D25982B7C9902C084E001C080E057
:1007C000892B7D9902C038E001C030E0832B7E99EF
:1007D00002C020E101C020E0822B9FB19095991FBB
:1007E0009927991F9295990F907E892B0FC0809120
:1007F0000101811149C080E40E94E002809301015F
:10080000882379F1B12C0E9402038B2DF80190818D
:10081000981719F08083C09200010E942503219649
:100820000F5F1F4FCE30D10509F076CF80910001C8
:10083000882361F1815080930001882339F08FE98A
:100840009FE00197F1F700C0000020C0A3E4B1E0F1
:10085000E5E3F1E0CF01825F91919D938E13FCCF90
:1008600015C083E10E940A03809301018111CACF60
:1008700081E40E94E002809301018111C3CF0E94B4
:100880001B03B82EB094BFCF80E0C0CF0E9470048D
:1008900081E0DF91CF911F910F91FF90EF90DF905A
:1008A000CF90BF900895E82FF0E0ED5BFE4F808180
:1008B000089508950F931F93CF93DF93C3E4D1E07E
:1008C00010E00C2F025F899190E00E94251C180F08
:1008D0000C13F9CF812FDF91CF911F910F910895C4
:1008E0000C94630556985E9825982D9826982E9816
:1008F00027982F988FEF90E090938900809388003D
:1009000090938B0080938A0090938D0080938C004D
:10091000259A2D9A2FEF80E792E021508040904059
:10092000E1F700C00000269A2E9A2FEF80E792E0B0
:10093000215080409040E1F700C00000279A2F9A94
:100940002FEF80E792E0215080409040E1F700C017
:10095000000025982D982FEF80E792E021508040ED
:100960009040E1F700C0000026982E982FEF80E716
:1009700092E0215080409040E1F700C000002798AD
:100980002F9856985E9825982D9826982E982798F7
:100990002F98089589EA8093800089E080938100F0
:1009A00024982C983F988AB18F748AB96E98479A88
:1009B0008BB1806B8BB9769A0E9472040C9462059D
:1009C00080E2809301018091510181110EC00E944B
:1009D000DA0281E0809351012FEF83ED90E3215003
:1009E00080409040E1F700C0000080E40E94E002F7
:1009F0008093010181112EC00E940A03809301019E
:100A0000811128C00E940A0380930101811122C034
:100A10008FE30E940A038093010181111BC00E9491
:100A2000020380E40E94E00280930101811112C060
:100A30008CE00E940A038093010181110BC00E9487
:100A40000A0380930101811105C08FE30E940A030C
:100A5000809301010E940203809101010895FC012D
:100A60006B3079F018F46A3031F01DC06C3079F0D9
:100A70006D3099F018C08281811118C08CE291E02C
:100A800008958281811115C08EE191E008958281DF
:100A9000811112C084E191E00895828181110FC01B
:100AA0008AE091E0089580E090E008958FE291E07F
:100AB000089581E291E0089589E191E008958FE041
:100AC00091E008950895CF936091BE017091BF01A8
:100AD0008091C0019091C1010E94311CC82F56988D
:100AE0005E9825982D9826982E9827982F988FE015
:100AF00090E0909389008093880090938B0080937E
:100B00008A0090938D0080938C00CC2329F0C13013
:100B100029F4C093520102C01092520180915201F7
:100B2000813011F4279A2F9A0E946810867011F074
:100B3000259A2D9AC23041F40E94AE1A811104C048
:100B400027982F98269A2E9AE0910E01F0910F0186
:100B50008081982F927259F08D7D49F48FEF90E04B
:100B60009093890080938800259A2D9A08C00E944E
:100B7000DB1B827221F00E94811A882379F3CF91C6
:100B8000089581E0089581E008950C94C3050895C7
:100B90000F931F93CF93DF938C01FC01C081D18110
:100BA000CE010E942A1ABE010E947106EC01B80112
:100BB0000E94C505882309F48DC0F801828188232D
:100BC00009F44AC080915E0181111FC0C431F0E573
:100BD000DF0709F051C00E94C70581E080935E01E4
:100BE0000E94C91C90935D0180935C011092550195
:100BF000109257011092560110925901109258010B
:100C000010925B0110925A0165C080915C01909135
:100C10005D010E94D51C883C910570F480915501BE
:100C2000E82FF0E0EE0FFF1FEA5AFE4FD183C0839A
:100C30008F5F809355014EC0C43880E5D80721F0FE
:100C4000C538D04501F13AC0F8018281882341F0CE
:100C50001092530182E01EC0C438E0E5DE0759F56A
:100C600080915301811106C086E20E94841186E2C0
:100C70000E944C1282E01CC0C438F0E5DF0741F34B
:100C8000C538D045D9F4F8018281882331F010921B
:100C9000540180E20E949B121DC080915401811179
:100CA00006C087E20E94841187E20E944C1280E213
:100CB0000E94A2120FC0C538D04529F381E080936D
:100CC000530180935401C801DF91CF911F910F917F
:100CD0000C94C10580E0DF91CF911F910F91089591
:100CE000089596E0799FF001112494E5899FE00D25
:100CF000F11D1124E60FF11DEE0FFF1FEE5BFE4FFD
:100D0000859194910895880F991FFC01E654F04055
:100D1000859194910895880F991FFC01E65CFE4F20
:100D20008591949108950F931F93CF93DF93EC01D6
:100D3000811520E3920750F5C11580E2D80708F02D
:100D4000C3C0CB3BD10590F4C83AD10508F06AC0C6
:100D5000C53AD10508F05BC0C430D10508F0D0C158
:100D6000219709F0CAC101E010E00AC2CF3FD105C6
:100D700011F008F0C5C1C03FD10508F0A2C0CE01F6
:100D8000805E9109089708F4BBC1B7C1C13090E5F6
:100D9000D90709F4A2C020F5C0318FE4D80770F458
:100DA000C11590E4D90708F094C0C11521E3D2071A
:100DB00008F0A3C1DD278E01106CE2C1C115D0453A
:100DC00009F09BC10E9431158FEF94E32CE0815014
:100DD00090402040E1F700C000000E94241DD0C1D7
:100DE000C11597E5D90758F4C03121E5D20708F0BD
:100DF0001CC1C43180E5D80708F475C07EC1CE019E
:100E000090578115904108F078C1DF7073C1C53AE1
:100E1000D10509F477C1C63AD10509F076C102E8D7
:100E200010E4AEC1C83AD10509F472C1C93AD1057E
:100E300009F471C1CA3AD10509F470C1CB3AD105A0
:100E400009F46FC1CC3AD10509F46EC1CD3AD10590
:100E500009F46DC1C03BD10509F46CC1CE3AD1058E
:100E600009F46BC1CF3AD10509F46AC1C13BD10580
:100E700009F469C1C23BD10509F468C1C33BD1057E
:100E800009F467C1C43BD10509F466C1C53BD1056E
:100E900009F465C1C63BD10509F464C1C73BD1055E
:100EA00009F463C1C83BD10509F462C1C93BD1054E
:100EB00009F461C1CA3BD10509F460C100E014E442
:100EC0005FC18E0110655CC1CE019F700E948B06D0
:100ED00058C1DF708E01106A53C18091E0018160BA
:100EE0008093E0014DC10E94C91E811102C00E9481
:100EF000AF1E0E94E61E90E09093010280930002D4
:100F0000C23080E5D80721F480910002816086C05C
:100F1000C43090E5D90721F48091000282607EC040
:100F2000C63020E5D20721F480910002846076C0AB
:100F3000C83080E5D80719F48091000227C0CA3074
:100F400090E5D90721F480910002806167C0CC3020
:100F500020E5D20721F48091000280625FC0CE308C
:100F600080E5D80721F480910002806457C0C03129
:100F700090E5D90721F48091000280684FC0C2310A
:100F800020E5D20729F4809100028460886046C081
:100F9000C33080E5D80721F4809100028E7F3EC0E7
:100FA000C53090E5D90721F4809100028D7F36C0CD
:100FB000C73020E5D20721F4809100028B7F2EC03C
:100FC000C93080E5D80719F48091000226C0CB30E3
:100FD00090E5D90721F4809100028F7E1FC0CD30AB
:100FE00020E5D20721F4809100028F7D17C0CF3019
:100FF00080E5D80721F4809100028F7B0FC0C131BA
:1010000090E5D90721F4809100028F7707C0C331A2
:10101000D04531F4809100028B7F877F809300025E
:10102000809100020E94EA1EABC08D2F99278F701D
:10103000992781309105D9F49E012370332702C08E
:10104000880F991F2A95E2F79C688E0144E0000FF3
:10105000111F4A95E1F700271370802B912B53E065
:10106000CC0FDD1F5A95E1F7C076DD272FC0823007
:10107000910531F4DC2FCC278E01016F106A80C0FE
:101080008330910569F4CE018370992701E010E067
:1010900002C0000F111F8A95E2F7C8019C680FC0BB
:1010A00084309105B9F4CE018370992701E010E0F6
:1010B00002C0000F111F8A95E2F7C8019A6823E069
:1010C000CC0FDD1F2A95E1F7C07ED7708C010C2B69
:1010D0001D2B56C08530910531F4DC2FCC278E01B5
:1010E000046F106A4DC0069709F04AC0CF71DD2722
:1010F000DC2FCC278E01106243C000E010E040C01E
:101100008E013EC001E810E43BC003E810E438C0A3
:1011100002EE14E435C009EE14E432C00AEE14E421
:101120002FC005EB14E42CC006EB14E429C007EB38
:1011300014E426C00CEC14E423C00DEC14E420C02D
:1011400003E815E41DC00AE815E41AC002E915E435
:1011500017C004E915E414C001E216E411C003E26B
:1011600016E40EC004E216E40BC005E216E408C063
:1011700006E216E405C007E216E402C00AE216E43D
:10118000C801DF91CF911F910F91089596E0799F4B
:10119000F001112494E5899FE00DF11D1124E60F63
:1011A000F11DEE0FFF1FEE5BFE4F85919491803E87
:1011B0009105E0F4803C910558F58133910509F4DF
:1011C0006FC048F48932910509F463C08A329105F1
:1011D00009F46DC072C089339105E9F08238910538
:1011E000D1F08533910509F44DC067C0833E910568
:1011F00081F138F4803E9105B9F0823E9105D9F035
:101200005CC0863E910561F1873E9105A1F155C014
:101210000E94830608952091000220FD02C021FF54
:101220004CC080EE90E049C08091000280FFF9CF71
:1012300089E390E042C08091000282FF0EC080915D
:10124000000284FF03C080E090E037C083EE90E0AE
:1012500034C08091000282FFF2CF82EE90E02DC078
:101260008091000283FF0BC08091000284FDEBCFD0
:1012700087EE90E022C08091000283FFF5CF86EEDA
:1012800090E01BC08091000285FF07C089E290E0DA
:1012900014C08091000285FFF9CF85E390E00DC076
:1012A0008091000286FF07C08AE290E006C080912C
:1012B000000286FFF9CF81E390E00E949306089533
:1012C00008950C94600980916F010895CF93DF9386
:1012D00000D01F92CDB7DEB79C018091F70184301A
:1012E00019F593E099833B832A839093E9008FEF6C
:1012F0009091E800815095FD06C095ED9A95F1F723
:1013000000008111F5CF8091E80085FF0DC040E01D
:1013100050E063E070E0CE0101960E94D00B809116
:10132000E8008E778093E8000F900F900F90DF9188
:10133000CF910895CF93DF9300D01F92CDB7DEB742
:101340002091F701243021F522E029839B838A83B1
:1013500083E08093E9008FEF9091E800815095FD44
:1013600006C095ED9A95F1F700008111F5CF8091B7
:10137000E80085FF0DC040E050E063E070E0CE0182
:1013800001960E94D00B8091E8008E778093E80050
:101390000F900F900F90DF91CF9108952091F7015A
:1013A0002430F1F422E02093E9002FEF3091E8009F
:1013B000215035FD06C035ED3A95F1F700002111B9
:1013C000F5CF2091E80025FF0BC040E050E065E03C
:1013D00070E00E94D00B8091E8008E778093E80047
:1013E0000895CF93DF93EC019091F701943009F0C9
:1013F00046C080910C018823D9F080910D0188238B
:10140000B9F09093E9008FEF9091E800815095FD3D
:1014100006C095E19A95F1F700008111F5CF809112
:10142000E80085FF2CC040E050E060E170E017C0AC
:1014300081E08093E9008FEF9091E800815095FD65
:1014400006C095ED9A95F1F700008111F5CF8091D6
:10145000E80085FF14C040E050E068E070E0CE0195
:101460000E94D00B8091E8008E778093E80080E1A5
:10147000FE01AFE5B1E001900D928A95E1F7DF91B1
:10148000CF9108958091F601811109C00E94650DE8
:101490000E94C20D8091E20084608093E200089572
:1014A0001092F601089508950C9459230E94BA1CD5
:1014B0000E945F230E9468100C94610942E061EC75
:1014C00081E00E94DF0C42E061EC82E00E94DF0CD0
:1014D00042E061EC83E00E94DF0C42E161EC84E0D9
:1014E0000C94DF0C8091F901833009F455C030F47D
:1014F000813071F0823009F48EC008958A3009F489
:101500007AC08B3009F460C0893009F09CC020C0DB
:101510008091F801813A09F096C08091E800877FB8
:101520008093E8008091FC019091FD01892B21F4CA
:1015300060E18FE591E003C060E080E090E070E062
:101540000E941B0C8091E8008B778093E80008953F
:101550008091F801813209F076C08091FC01909170
:10156000FD01009719F0039709F06DC08091E80024
:10157000877F8093E8008091E80082FD05C080911C
:10158000F7018111F8CF5FC08091F10080936F0166
:101590008091E8008B7753C08091F801813A09F07F
:1015A00052C08091FC019091FD01892B09F04BC044
:1015B0008091E800877F8093E8008091E80080FFB9
:1015C000FCCF80910C0136C08091F8018132D9F5B1
:1015D0008091FC019091FD01892BA9F58091E80093
:1015E000877F8093E8000E94140D8091FA01809318
:1015F0000C010C9431158091F801813221F5809114
:10160000E800877F8093E8000E94140D8091FB0121
:101610008093700108958091F801813AA1F480913E
:10162000E800877F8093E8008091E80080FFFCCF8E
:10163000809170018093F1008091E8008E77809313
:10164000E8000C94140D089584B7877F84BF88E167
:101650000FB6F89480936000109260000FBE90E087
:1016600080E80FB6F89480936100909361000FBEFC
:101670000E94B7100E94650D0E94C20D8091E20089
:1016800084608093E20078940E9448100E94B91010
:1016900082E091E00E9463100E9447238091F7014D
:1016A000853069F40E94811C8091F5018823B1F393
:1016B0000E94AC1C882391F30E94BA0BEFCF0E94CA
:1016C000BF10ECCF292F332723303105C9F064F444
:1016D0002130310581F02230310509F043C08DE61B
:1016E00090E02EE633E042C021323105F1F02232A3
:1016F000310541F137C082E190E02BED33E036C097
:1017000099278130910541F08230910541F0892B74
:1017100049F5EAE6F3E005C0E2E5F3E002C0EAE3FA
:10172000F3E0849190E09F0121C06430D8F4E62F6B
:10173000F0E0EE0FFF1FEE5DFE4F2081318189E06A
:1017400090E014C0643070F470E0FB01EE0FFF1FF6
:10175000E65EFE4F20813181FB01EA5EFE4F808113
:1017600090E004C080E090E020E030E0FA013183B6
:101770002083089580E189BD82E189BD09B400FE1E
:10178000FDCF8091D8008F7D8093D8008091E000BC
:1017900082608093E0008091E00081FDFCCF08959D
:1017A000CF92DF92EF92FF920F931F93CF93DF932D
:1017B000EC018B016A010E94330D811133C0C11409
:1017C000D10439F0F60180819181081B190BC80FF3
:1017D000D91FE12CF12C0115110519F18091E800B8
:1017E00085FD16C08091E8008E778093E800C114D3
:1017F000D10449F0F60180819181E80EF91EF18251
:10180000E08285E00FC00E94330D882321F30AC0D7
:1018100089918093F10001501109FFEFEF1AFF0A3F
:10182000DACF80E0DF91CF911F910F91FF90EF9081
:10183000DF90CF9008952091FE013091FF0126178F
:10184000370748F06115710539F42091E8002E77CB
:101850002093E80001C0B90140E061157105A9F1CC
:101860002091F701222309F443C0253009F442C036
:101870002091E80023FD40C02091E80022FD32C005
:101880002091E80020FFE9CF4091F3002091F20081
:1018900030E0342BFC01CF016115710559F028307F
:1018A000310540F481918093F100615071092F5FFF
:1018B0003F4FF1CF41E02830310509F040E0209161
:1018C000E8002E772093E800C8CF4111C9CF0AC0A5
:1018D0008091F701882361F0853061F08091E80004
:1018E00083FD0AC08091E80082FFF2CF80E0089576
:1018F00082E0089583E0089581E008952091FE013B
:101900003091FF012617370748F06115710539F44A
:101910002091E8002E772093E80001C0B901FC0176
:1019200020E06115710591F18091F701882309F498
:1019300040C0853009F43FC08091E80083FD3DC080
:101940008091E80082FD2FC08091E80080FFE9CF00
:101950002091F3008091F20090E0922B61157105C7
:1019600059F08830910540F424912093F10031968C
:10197000615071090196F2CF21E0089709F020E04B
:101980008091E8008E778093E800CBCF2111CCCFF7
:101990000AC08091F701882361F0853061F0809161
:1019A000E80083FD0AC08091E80082FFF2CF80E06A
:1019B000089582E0089583E0089581E00895982FC6
:1019C000973058F59093E900981739F07091EC0032
:1019D0002091ED005091F00003C0242F762F50E0AD
:1019E00021FF19C03091EB003E7F3093EB00309126
:1019F000ED003D7F3093ED003091EB00316030938E
:101A0000EB007093EC002093ED005093F0002091D8
:101A1000EE0027FF07C09F5FD3CF8F708093E90050
:101A200081E0089580E008958091F80187FF11C05A
:101A30008091E80082FD05C08091F7018111F8CF07
:101A400011C08091E8008B770BC08091F70188234B
:101A500049F08091E80080FFF8CF8091E8008E7710
:101A60008093E80008952091E4003091E50095E628
:101A70004091EC00842F817040FF22C08091E800EB
:101A800080FD1CC08091F701882391F0853091F092
:101A90008091EB0085FD10C04091E4005091E5007D
:101AA0004217530729F39A01915011F784E00895E2
:101AB00082E0089583E0089581E0089580E008952C
:101AC0004091E80042FFDECF08950E94D30D0E94AE
:101AD000DB0DE0EEF0E0808181608083E8EDF0E0F6
:101AE00080818F77808319BCA7EDB0E08C918E7FC9
:101AF0008C9380818F7E80831092F60108950F93DE
:101B00001F93CF93DF930E94D30D0E94DB0DC8ED8E
:101B1000D0E088818F7788838881806888838881F6
:101B20008F7D888319BC1092F7011092F3011092F7
:101B3000F5011092F40100EE10E0F80180818B7F36
:101B4000808388818160888342E060E080E00E9439
:101B5000DF0CE1EEF0E080818E7F8083E2EEF0E04A
:101B6000808181608083808188608083F8018081AA
:101B70008E7F8083888180618883DF91CF911F91E0
:101B80000F910895E8EDF0E080818F7E8083E7ED8E
:101B9000F0E080818160808384E082BF81E0809377
:101BA000F6010C947F0DE8EDF0E080818E7F80835C
:101BB0001092E20008951092DA001092E100089568
:101BC0001F920F920FB60F9211242F933F934F93B2
:101BD0005F936F937F938F939F93AF93BF93EF9395
:101BE000FF938091E10082FF0BC08091E20082FFB1
:101BF00007C08091E1008B7F8093E1000E94471035
:101C00008091DA0080FF1FC08091D80080FF1BC048
:101C10008091DA008E7F8093DA008091D90080FF76
:101C20000DC080E189BD82E189BD09B400FEFDCF10
:101C300081E08093F7010E94420A05C019BC10920E
:101C4000F7010E94500A8091E10080FF19C0809145
:101C5000E20080FF15C08091E2008E7F8093E20059
:101C60008091E20080618093E2008091D8008062E0
:101C70008093D80019BC85E08093F7010E94540A34
:101C80008091E10084FF30C08091E20084FF2CC08D
:101C900080E189BD82E189BD09B400FEFDCF80915C
:101CA000D8008F7D8093D8008091E1008F7E809353
:101CB000E1008091E2008F7E8093E2008091E2005B
:101CC00081608093E2008091F301882311F084E029
:101CD00007C08091E30087FD02C081E001C083E07E
:101CE0008093F7010E94560A8091E10083FF29C08A
:101CF0008091E20083FF25C08091E100877F80937F
:101D0000E10082E08093F7011092F3018091E100FD
:101D10008E7F8093E1008091E2008E7F8093E200CD
:101D20008091E20080618093E20042E060E080E028
:101D30000E94DF0C8091F00088608093F0000E9488
:101D4000530AFF91EF91BF91AF919F918F917F9136
:101D50006F915F914F913F912F910F900FBE0F9018
:101D60001F9018951F920F920FB60F9211242F9368
:101D70003F934F935F936F937F938F939F93AF9313
:101D8000BF93CF93DF93EF93FF93C091E900CF70A0
:101D90008091EC00D82FD17080FDD0E81092E9003E
:101DA0008091F000877F8093F00078940E94F60E77
:101DB0001092E9008091F00088608093F000CD2BB4
:101DC000CF70C093E900FF91EF91DF91CF91BF9168
:101DD000AF919F918F917F916F915F914F913F91C3
:101DE0002F910F900FBE0F901F9018951F93CF93B8
:101DF000DF93CDB7DEB7AA970FB6F894DEBF0FBE5C
:101E0000CDBFE8EFF1E088E08E0F9091F100919363
:101E10008E13FBCF0E94720A8091E80083FF1FC1DE
:101E20008091F8019091F901492F50E04A30510515
:101E300008F015C1FA01EA5AFF4F0C94E1248038EA
:101E400081F0823809F00BC18091FC018F70809382
:101E5000E9008091EB0085FB882780F91092E9006A
:101E600006C08091F4019091F501911182609091EA
:101E7000E800977F9093E8008093F1001092F100C2
:101E8000C8C0282F2D7F09F0EAC0882319F08230BE
:101E900061F0E5C08091FA01813009F0E0C0933033
:101EA00009F080E08093F5012BC08091FA01811147
:101EB00027C08091FC018F7009F4D1C08093E900A4
:101EC0002091EB0020FF1CC0933021F48091EB00A7
:101ED000806214C09091EB0090619093EB0021E040
:101EE00030E0A90102C0440F551F8A95E2F74093E4
:101EF000EA001092EA008091EB0088608093EB008A
:101F00001092E9008091E800877F86C08111A7C008
:101F10001091FA011F778091E3008078812B8093E4
:101F2000E3008091E800877F8093E8000E94140D11
:101F30008091E80080FFFCCF8091E300806880936F
:101F4000E300111102C082E001C083E08093F70139
:101F500086C08058823008F082C08091FA0190914A
:101F6000FB018C3D53E0950779F583E08A838AE293
:101F700089834FB7F894DE01139620E03EE051E2EA
:101F8000E32FF0E050935700E49120FF03C0E29567
:101F9000EF703F5FEF708E2F90E0EA3010F0C79641
:101FA00001C0C0968D939D932F5F243149F74FBF99
:101FB0008091E800877F8093E8006AE270E0CE01BC
:101FC00001960E941B0C14C0AE014F5F5F4F6091E1
:101FD000FC010E94620BBC01009709F440C0909183
:101FE000E800977F9093E80089819A810E947E0C97
:101FF0008091E8008B778093E80031C0803879F5D4
:102000008091E800877F8093E8008091F3018093BE
:10201000F1008091E8008E778093E8000E94140D13
:102020001EC081111CC09091FA019230C0F48091C1
:10203000E800877F8093E8009093F3010E94140DDD
:102040008091F301811106C08091E30087FD02C0F9
:1020500081E001C084E08093F7010E945E0A8091D4
:10206000E80083FF0AC08091E800877F8093E80042
:102070008091EB0080628093EB00AA960FB6F894F3
:10208000DEBF0FBECDBFDF91CF911F9108950895A0
:10209000CF938091F7018823A1F0C091E900CF7020
:1020A0009091EC00892F817090FD80E8C82B1092F0
:1020B000E9008091E80083FD0E94F60ECF70C09386
:1020C000E900CF910895909376018093750108956A
:1020D000E0917501F0917601309721F00190F08147
:1020E000E02D099480E00895E0917501F09176016A
:1020F000309721F00280F381E02D09940895E0915A
:102100007501F0917601309721F00480F581E02D82
:1021100009940895209173013091740182179307F7
:1021200071F09093740180937301E0917501F091C7
:102130007601309721F00680F781E02D099408950B
:1021400020917101309172018217930771F0909381
:10215000720180937101E0917501F09176013097E1
:1021600021F00084F185E02D0994089508950C94E0
:10217000B6100E94C01C0E944D030C94821D9F92B9
:10218000AF92BF92CF92DF92EF92FF920F931F9385
:10219000CF93DF9300D000D000D0CDB7DEB70E9440
:1021A00065030DE010E0AA24A394B12C902E802F9B
:1021B0000E945304980128583E4F6901F901F080AC
:1021C000F826A1F40150110988F78FEF89838A83DB
:1021D0001B820E94C91C8160782F9D838C8349815A
:1021E0005A816B818D810E9456112FC09091E00120
:1021F00091FF04C08E830E9459048E8125E030E057
:10220000A501022E01C0440F0A94EAF7E42E4F21E3
:10221000C1F029839A828E2191E009F490E09B839A
:102220000E94C91C8160782F9D838C8349815A81CB
:102230006B818D810E945611F6018081E826E08233
:1022400004C021503109E0F6BDCF0E9469201091F1
:1022500077010E9468101817B9F00E9468108093E7
:10226000770126960FB6F894DEBF0FBECDBFDF9183
:10227000CF911F910F91FF90EF90DF90CF90BF9083
:10228000AF909F900C94610926960FB6F894DEBF2C
:102290000FBECDBFDF91CF911F910F91FF90EF90B7
:1022A000DF90CF90BF90AF909F900895CF93DF9332
:1022B000CDB7DEB72B970FB6F894DEBF0FBECDBFFC
:1022C0004F83588769877A878B87DE01119686E06E
:1022D000FD0111928A95E9F785E0FE01379601909C
:1022E0000D928A95E1F749815A816B817C818D81BC
:1022F0009E810E94CF172B960FB6F894DEBF0FBEBB
:10230000CDBFDF91CF910895CF93882309F4C2C048
:10231000C82F823859F40E94681081FDBBC089E340
:102320000E94121B0E94EF1B89E30CC0833879F4D2
:102330000E94681080FDAEC083E50E94121B0E94BF
:10234000EF1B83E50E94541BCF910C94EF1B843844
:1023500059F40E94681082FD9DC087E40E94121B00
:102360000E94EF1B87E4EECF8CEF8C0F813A48F48C
:102370008C2F0E94AC2281118DC08C2F0E94121BC9
:10238000E3CF80E28C0F883048F4C77081E001C051
:10239000880FCA95EAF70E949B1BD6CF8BE58C0F5E
:1023A000833078F4C53A29F0C63A31F083E890E0FA
:1023B00005C081E890E002C082E890E0CF910C94E3
:1023C0008A1088E58C0F833108F064C0C83A39F16F
:1023D000C93A41F1CA3A49F1CB3A51F1CC3A59F1F3
:1023E000CD3A61F1C03B69F1CE3A71F1CF3A79F162
:1023F000C13B81F1C23B89F1C33B91F1C43B99F1EF
:10240000C53BA1F1C63BA9F1C73BB1F1C83BB9F14E
:10241000C93BC1F1CA3BC9F180E090E038C082EE0F
:1024200090E035C089EE90E032C08AEE90E02FC097
:1024300085EB90E02CC086EB90E029C087EB90E024
:1024400026C08CEC90E023C08DEC90E020C083E8A7
:1024500091E01DC08AE891E01AC082E991E017C0BE
:1024600084E991E014C081E292E011C083E292E03D
:102470000EC084E292E00BC085E292E008C086E2E2
:1024800092E005C087E292E002C08AE292E0CF913A
:102490000C94A010CF910895882309F44BC0823882
:1024A00059F40E94681081FF45C089E30E94121B05
:1024B0000E94EF1B89E30CC0833871F40E946810FE
:1024C00080FF38C083E50E94121B0E94EF1B83E54A
:1024D0000E94541B0C94EF1B843859F40E9468101E
:1024E00082FF28C087E40E94121B0E94EF1B87E432
:1024F000EFCF9CEF980F913A58F390E2980F9830F5
:1025000050F4877091E001C0990F8A95EAF7892FFE
:102510000E94A11BDFCF9BE5980F933020F480E051
:1025200090E00C948A10885A833120F480E090E087
:102530000C94A0100895882321F00E949B1B0C94FA
:10254000EF1B0895882321F00E94A11B0C94EF1B20
:1025500008958F929F92AF92BF92DF92EF92FF9277
:102560000F931F93CF93DF937C01D62FC72FFC01CE
:102570000281158112951F700E94AE1A882319F0EE
:1025800082E00E94F01A01110E94B81B0E940B1BEE
:10259000882379F0002369F080E28D0F883048F0BD
:1025A00082E00E94F01A0E940B1B91E0D82ED926DF
:1025B00001C0D12CEC2FE295EF70F0E0E05AFF4F14
:1025C0000C94E1248C2F807FCF70882311F0C2956A
:1025D000C07F002389F0CC2309F4C4C180E28D0FB1
:1025E000883020F48C2F0E949B1B03C08C2F0E94EC
:1025F000AB1B0E94EF1BB6C18D2F0E944C12CC2347
:1026000009F4CAC1D05E8C2FD83018F40E94A11BE7
:1026100002C00E94B11B0E94EF1BBEC18C2F807FA5
:10262000CF70803211F0C295C07FDD2319F0D13018
:1026300029F12DC0002381F0112369F1113021F41B
:102640008C2F0E94CB1BA8C1123029F50E94D41BED
:102650008C2F0E947B1A1FC0112369F0113041F4A6
:102660000E94981B8C2309F497C10E947E1A03C014
:10267000123009F491C10E94D41B11C0002321F033
:10268000123008F089C107C0111186C108C00023AB
:1026900021F0111167C18C2FF1C011116AC18C2F6B
:1026A000F3C08C2F86958695837090E0009719F083
:1026B000019761F071C1002321F08D2F9C2F937041
:1026C00002C080E090E00E948A1066C1002321F0E1
:1026D0008D2F9C2F937002C080E090E00E94A0108C
:1026E0005BC18D2F002319F00E94711F02C00E9450
:1026F000D91F0E945E2050C18C2F837009F050C0FA
:1027000001114AC18D2F829586958770880F880F99
:102710009D2F9F70892E912CA12CB12C082E04C0C6
:10272000880C991CAA1CBB1C0A94D2F7D4FF14C0B5
:102730000FE010E020E030E0B901A80104C0440F30
:10274000551F661F771F8A95D2F7CB01BA01609596
:1027500070958095909503C060E070E0CB01C695C0
:10276000C695C370D0E0C230D10561F0C330D10549
:1027700081F0682979298A299B29219771F00E9483
:1027800017190AC1682979298A299B290E943319B6
:1027900003C10E941719C501B4010E94FB18FCC0B7
:1027A000002319F08C2F817001C08695882309F4CD
:1027B000F3C08D2F829586958770880F880F9D2F87
:1027C0009F70892E912CA12CB12C082E04C0880C4E
:1027D000991CAA1CBB1C0A94D2F7D4FF14C00FE0AA
:1027E00010E020E030E0B901A80104C0440F551FFB
:1027F000661F771F8A95D2F7CB01BA016095709555
:102800008095909503C060E070E0CB01C695C695B9
:10281000C3704C2F50E04230510569F043305105F0
:1028200089F0682979298A299B294130510571F05D
:102830000E94F119B1C0682979298A299B290E942F
:102840000D1AAAC00E94F119C501B4010E94D51940
:10285000A3C08D2F90E0FC01E05EF109E531F105A8
:1028600008F07BC0E059FF4F0C94E124DF708C2FFF
:102870008F71002331F00E946E198D2F0E949B12E0
:102880008BC00E948F198D2F0E94A21285C0002339
:1028900039F0111181C08C2F8F710E94B4197CC046
:1028A000123008F079C0F7CF002339F08C2F8F71E8
:1028B0000E946E1971C00023C9F38C2F8F710E9482
:1028C0008F196AC0002329F08C2F8F710E9459192B
:1028D00063C00E944F1960C00023B9F00E94781AAB
:1028E0000E94A11B0E94AA1A843029F40E94E91AAE
:1028F0008C2F8F7162C0123008F06CC0CF718C2F9A
:102900000E946E1963E08C2F0DC00E94781A0E94FD
:102910009B1B1230A0F00E94E91A0E947E1A64E00C
:102920008C2F8F71DF91CF911F910F91FF90EF90BE
:10293000DF90BF90AF909F908F900C94D91A81E058
:10294000DF91CF911F910F91FF90EF90DF90BF909B
:10295000AF909F908F900C94F01A002339F01123C0
:1029600009F4A4CF8D2F0E94841116C0112309F4FD
:10297000A4CF8D2F0E944C120FC04C2F4F706D2F83
:10298000C7010E942F050E94731806C04C2F4F707C
:102990006D2FC7010E947006DD20E1F00E94AA1A87
:1029A00080FD18C0F70112820E94A41A0E946E19BD
:1029B000C7010E94F6140E94A41ADF91CF911F91C3
:1029C0000F91FF90EF90DF90BF90AF909F908F900E
:1029D0000C948F19DF91CF911F910F91FF90EF9081
:1029E000DF90BF90AF909F908F9008950F931F93AB
:1029F000CF93DF93EC01888199812B813C81232B3C
:102A0000B9F09F3F11F48F3F99F0CE010E94C805A5
:102A1000882371F0688179818A810E94741A8C01FF
:102A20000E94291A0E94F018B801CE010E94A91232
:102A3000DF91CF911F910F9108950E94B81B0E94C2
:102A4000C81B0E948A1B0E94EF1B0E940F210E943C
:102A50005E2080E090E00E948A1080E090E00C947C
:102A6000A0100E94A81B0C941D150E94691A292F02
:102A700022952F7030E02C3031054CF42A3031058E
:102A80006CF42250310922303105A8F407C02C30F3
:102A9000310569F02F30310551F00DC0803F69F0EC
:102AA00018F4803E40F409C0843F29F406C093FB2B
:102AB000882780F9089580E0089581E00895CF93F4
:102AC000DF9300D000D01F92CDB7DEB70F900F90EC
:102AD0000F900F900F90DF91CF910895CF93DF93D8
:102AE00000D000D000D0CDB7DEB726960FB6F89450
:102AF000DEBF0FBECDBFDF91CF9108951F93CF935F
:102B0000DF93C091860116E080918701C81799F084
:102B1000D0E01C9FF0011D9FF00D1124E857FE4FDF
:102B20004081518162817381848195810E946E15FB
:102B30002196C770E9CFDF91CF911F910895409101
:102B4000B8015091B9016091BA017091BB018091B7
:102B5000BC019091BD010C946E158091BD018295D0
:102B60008F7009F054C08091BA01882309F44FC0D6
:102B700080918601A09187016091B8017091B9019F
:102B80004091BB015091BC01B6E08A1709F43FC0E7
:102B900090E041155105C1F17F3F11F46F3FA1F164
:102BA000B89FF001B99FF00D1124E857FE4F218125
:102BB00072132AC02081621327C02281211124C0F0
:102BC000238134812417350710F421503109241B47
:102BD000350B283C3105C0F42091BD012F702061D8
:102BE0002093BD0126E0289FF001299FF00D1124BC
:102BF000E357FE4F80818F708061808388EB91E086
:102C00000E94F6140C947E1501968770BECF08952D
:102C1000CF92DF92EF92FF920F931F93CF93DF93A8
:102C2000CDB7DEB762970FB6F894DEBF0FBECDBF4B
:102C30008C0185E0F801DE011D9601900D928A95C8
:102C4000E1F7D8014C9111965C91119712966C9115
:102C500012971396CD90DC9014973091B801709133
:102C6000B9018091BB019091BC01009709F46BC13F
:102C70007F3F19F43F3F09F466C1E090BA01EE20AE
:102C800009F4C0C02091BD01C816D90628F0F6018C
:102C9000E81BF90BCF0104C0809590958C0D9D1D0C
:102CA000FF24F394883C910578F0F12C207F09F003
:102CB000C6C07C2DD98AC88A89890E945F1588EB95
:102CC00091E00E94F614B1C0822F807F09F046C0C7
:102CD000751314C0341312C0611110C02F7020611D
:102CE0002093BD010E949F1588EB91E00E94F6148D
:102CF0008091BD01D80115968C932EC0CD2819F175
:102D00005F3F11F44F3FF9F0F62E61111CC0809126
:102D100086012091870136E0821709F45AC090E0BD
:102D2000389FF001399FF00D1124E857FE4F718153
:102D3000571306C07081471303C07281711103C01D
:102D400001968770E9CFF62E662309F418C18091A9
:102D5000BD0181608093BD01F12C11C1751308C0C4
:102D6000341306C0611104C08091BD01D801C3C0F5
:102D70004D875E878D859E856A8B0E9435156A8991
:102D80008823E1F16623D1F12091BD01822F829544
:102D90008F7090E0029774F08091B8019091B90122
:102DA00098878F831986DB86CA862C87CE01079683
:102DB0000E94F61486E0F801A8EBB1E001900D92B4
:102DC0008A95E1F70E94AD150E949F15FF24F394A8
:102DD000D6C04D875E878D859E850E94691A292FF2
:102DE00022952F7030E0223031050CF0BCC09F706E
:102DF00009F0B6C0805E883008F4C1C0C8010E94E6
:102E0000F614E4CFC816D90608F453C0F601E81B3F
:102E1000F90BCF01883C910508F450C0F12C7C2DB2
:102E2000D98AC88A89890E945F15E8EBF1E086E0BB
:102E3000DF011D928A95E9F70E949F15A0C07513C6
:102E400014C0341312C0611110C08091BD01F8018B
:102E50008583C8010E94F61486E0E8EBF1E0DF010B
:102E60001D928A95E9F7FE2C8AC04D875E878D8575
:102E70009E856A8B0E9435156A89882309F4BECF26
:102E8000662309F4BBCF2091BD01822F82958F70FC
:102E900090E002970CF48ECF8091B8019091B90127
:102EA0009A8389831B82DD82CC822E83CE01019698
:102EB0007FCF809590958C0D9D1DACCFF62E66230F
:102EC00009F49CCF75132EC034132CC02091BD0182
:102ED00020FD1FC0822F82958F70D9F0D8011596E2
:102EE0002C9315978F3049F08F5F982F9295907F94
:102EF000822F8F70892B15968C93C8010E94F6142F
:102F000086E0F801A8EBB1E001900D928A95E1F717
:102F100093CF86E0F801A8EBB1E001900D928A957D
:102F2000E1F72DC04D875E878D859E850E94351502
:102F3000811140CF8091BD0181608093BD01C801A6
:102F40000E94F6141CC0662309F458CF4D875E8793
:102F50008D859E850E943515882309F44FCF2ACF91
:102F6000811148CF0CC0243031050CF047CF9F7041
:102F700009F440CFF8019581907F09F03BCF8F2D68
:102F800062960FB6F894DEBF0FBECDBFDF91CF9132
:102F90001F910F91FF90EF90DF90CF9008951F93B6
:102FA000CF93DF93CDB7DEB72C970FB6F894DEBF83
:102FB0000FBECDBF4F83588769877A878B879C87E1
:102FC000CE0107960E940816882369F08F819885A4
:102FD0002A853B85232BF1F19F3F09F063C08F3F8A
:102FE00009F060C037C086E0FE013796DE01119619
:102FF00001900D928A95E1F76F817885EA85FB85CE
:10300000309741F17F3F11F46F3F21F1209187010B
:1030100030E0C9010196877099274091860150E000
:103020008417950709F447C069837A83FD83EC838D
:1030300096E0929FD001939FB00D1124A857BE4FE8
:10304000FE01319601900D929A95E1F780938701E8
:103050000E947E1516E08091860190918701891764
:10306000C1F1189FC001112488579E4F0E94081675
:10307000882379F1E09186011E9FF0011124E85721
:10308000FE4F4081518162817381848195810E94CC
:103090006E158091860190E0019687709927809344
:1030A0008601D9CF4F81588569857A858B859C8526
:1030B0000E946E15CFCF0E94311510928701109299
:1030C0008601E8EBF1E086E0DF011D928A95E9F7E1
:1030D000C1CF2C960FB6F894DEBF0FBECDBFDF91E7
:1030E000CF911F910895EF92FF920F931F93CF936B
:1030F000DF938C01009709F46CC0F12CEE24E3946B
:10310000E8012196F8018491843740F4843008F076
:1031100051C0813081F0823019F15BC0853709F4EC
:1031200044C0A8F19CE7980F903708F052C08F7701
:103130000E944C1241C00E5F1F4FFE01C49180E2FD
:103140008C0F883048F4C7708E2D01C0880FCA9547
:10315000EAF70E94BB1B14C08C2F0E9484112DC063
:103160000E5F1F4FFE01C49180E28C0F883058F42F
:10317000C7708E2D01C0880FCA95EAF70E94C11B47
:103180000E94EF1B1AC08C2F0E944C1216C00E5FBB
:103190001F4FFE01C491CC2381F08FE99FE001977E
:1031A000F1F700C00000C150F6CF0E5F1F4FFE01C7
:1031B000F49003C00E9484118E018F2D882309F49E
:1031C0009FCFEFE9FFE03197F1F700C00000815099
:1031D000F5CFDF91CF911F910F91FF90EF90089560
:1031E00008956093C2017093C3018093C4019093CA
:1031F000C5010C941D150F931F930091C2011091EE
:10320000C3012091C4013091C501DC01CB01802BA9
:10321000912BA22BB32B8093C2019093C301A09357
:10322000C401B093C5011F910F910C941D150F930C
:103230001F930091C2011091C3012091C4013091EC
:10324000C501DC01CB0180239123A223B32380930A
:10325000C2019093C301A093C401B093C5011F9113
:103260000F910C941D150F931F930091C2011091A3
:10327000C3012091C4013091C501DC01CB0180273D
:103280009127A227B3278093C2019093C301A093F3
:10329000C401B093C5011F910F910C941D1510929C
:1032A000BE011092BF011092C0011092C1010C9496
:1032B0001D1541E050E060E070E004C0440F551F70
:1032C000661F771F8A95D2F74093BE015093BF01C6
:1032D0006093C0017093C1010C941D1541E050E052
:1032E00060E070E004C0440F551F661F771F8A9589
:1032F000D2F78091BE019091BF01A091C001B09121
:10330000C101482B592B6A2B7B2B4093BE01509354
:10331000BF016093C0017093C1010C941D1541E081
:1033200050E060E070E004C0440F551F661F771F37
:103330008A95D2F740955095609570958091BE0121
:103340009091BF01A091C001B091C10148235923C0
:103350006A237B234093BE015093BF016093C00159
:103360007093C1010C941D1541E050E060E070E0E5
:1033700004C0440F551F661F771F8A95D2F78091AE
:10338000BE019091BF01A091C001B091C101482739
:1033900059276A277B274093BE015093BF01609352
:1033A000C0017093C1010C941D150F931F930091E0
:1033B000BE011091BF012091C0013091C101DC011B
:1033C000CB01802B912BA22BB32B8093BE0190932A
:1033D000BF01A093C001B093C1011F910F910C9444
:1033E0001D150F931F930091BE011091BF012091F5
:1033F000C0013091C101DC01CB0180239123A223C4
:10340000B3238093BE019093BF01A093C001B093FA
:10341000C1011F910F910C941D150F931F930091E3
:10342000BE011091BF012091C0013091C101DC01AA
:10343000CB0180279127A227B3278093BE019093C9
:10344000BF01A093C001B093C1011F910F910C94D3
:103450001D150895CF92DF92EF92FF920F931F9365
:10346000CF93DF938C01C090C201D090C301E09054
:10347000C401F090C5018091BE019091BF01A0915F
:10348000C001B091C101C82AD92AEA2AFB2ACFE19A
:10349000D0E0D701C6010C2E04C0B695A79597952C
:1034A00087950A94D2F780FF06C0B8018C2F0E943E
:1034B000C608019721F4219760F780E001C08C2FA6
:1034C000DF91CF911F910F91FF90EF90DF90CF9000
:1034D0000895CF93DF93EC010E942A1ABE010E9447
:1034E000C608DF91CF910895CB010E94691A089513
:1034F0008091CB0108958093CB0108951092CB0168
:1035000008950E94C91C2091C9013091CA018217F7
:10351000930750F00E94C91C2091C9013091CA0143
:10352000821B930B9C010AC00E94C91C2091C901F7
:103530003091CA0120953095280F391F81E0283B32
:103540003B4008F480E008958091C80185958595F9
:10355000859508958091C801877008950E94C91CBF
:103560002091C6013091C70182179307A8F00E94ED
:10357000C91C2091C6013091C701821B930B883B67
:103580009B4010F480E013C08091C80182FB882723
:1035900080F991E089270BC00E94C91C2091C601C7
:1035A0003091C70120953095820F931FE8CF81702D
:1035B000089598E0899F90011124262B2093C8013B
:1035C0000E946E190E94C91C9093C7018093C60186
:1035D00008951092C8011092C7011092C601089573
:1035E0002091C801809582238093C801982F9770FD
:1035F00089F430E0482F552747FD509524173507AB
:1036000049F08595859585950E948F191092C7017F
:103610001092C60108959091C801977081E009F455
:1036200080E0089590910C01992321F090910D0173
:10363000911109C020910E0130910F01F9013296CC
:103640009FEF40E01FC0982F9695969596959F30D6
:1036500050F5E0910E01F0910F01E90FF11D877017
:1036600021E030E0A90102C0440F551F8A95E2F71E
:10367000CA019181892B818308959F3F39F04F5F63
:103680004E3041F051915813F8CF0DC05111F7CF82
:10369000942FF5CF9F3F39F0F901E90FF11D97FD08
:1036A000FA9582830895089590910C01992321F051
:1036B00090910D01911109C020910E0130910F01DF
:1036C000F9013296205F3F4F1FC0982F969596952F
:1036D00096959F30F0F4E0910E01F0910F01E90F03
:1036E000F11D877021E030E0A90102C0440F551F91
:1036F0008A95E2F7CA018095918189238183089593
:103700003196E217F30729F090819813F9CF1082D0
:10371000F7CF089581E090E0E0910E01F0910F0164
:10372000E80FF91F1082019680319105A9F70895DD
:103730008091DF0108959091DF01892B8093DF0153
:10374000089580959091DF0189238093DF0108958A
:103750001092DF0108959091DE01892B8093DE01A4
:10376000089580959091DE0189238093DE0108956C
:103770001092DE0108959091DD01892B8093DD0187
:10378000089580959091DD0189238093DD0108954E
:103790001092DD0108958093CC010E94C91C909382
:1037A000CA018093C90108951092CC011092CA01F8
:1037B0001092C90108958091CC01089580910E0165
:1037C00090910F01FC0131969C01205F3F4F80E0FA
:1037D000919191118F5FE217F307D1F70895E0916E
:1037E0000E01F0910F018091DF018083E0910E01C5
:1037F000F0910F0190818091DE01892B8083E0910F
:103800000E01F0910F0190818091DD01892B808361
:103810008091CC01882399F00E94811A81110E9425
:10382000D41BE0910E01F0910F0190818091CC01A9
:10383000892B80830E94DE1B81110E94D41B809102
:103840000E0190910F010C94741020E0009739F054
:10385000AC0141505109842395232F5FF7CF822F6C
:103860000895CF92DF92EF92FF926C01EE24FF2435
:10387000C114D104E104F10421F0C701B60120E133
:1038800001C020E0C72ED82EE92EFF24C114D10498
:10389000E104F10419F0285FC701B6016B017C0156
:1038A00054E0F694E794D794C7945A95D1F7C1148D
:1038B000D104E104F10419F02C5FC701B6016B01DA
:1038C0007C0142E0F694E794D794C7944A95D1F7E7
:1038D000C114D104E104F10419F02E5FC701B6014F
:1038E000DC01CB01B695A79597958795892B8A2BF7
:1038F0008B2B09F02F5F822FFF90EF90DF90CF90FE
:1039000008958091F701843021F11092E10120E4C3
:1039100088E190E00FB6F894A895809360000FBE00
:103920002093600080E00E94610983B7817F8460FA
:1039300083BF83B7816083BF7894889583B78E7F78
:1039400083BF88E10FB6F894809360001092600006
:103950000FBE0895089508950E94AA1C0E94650351
:103960000E94AB1C0E945A0491E0811101C090E0BA
:10397000892F08950E9431150E9468100C946109E6
:1039800082E084BD93E095BD9AEF97BD80936E0071
:1039900008952FB7F8948091E2019091E301A091EE
:1039A000E401B091E5012FBF0895CF92DF92EF922D
:1039B000FF920F931F932FB7F8944091E20150911B
:1039C000E3016091E4017091E5012FBF6A017B0181
:1039D000EE24FF248C0120E030E0C016D106E20680
:1039E000F30610F4415051099A01281B390BC90103
:1039F0001F910F91FF90EF90DF90CF9008951F924D
:103A00000F920FB60F9211248F939F93AF93BF9392
:103A10008091E2019091E301A091E401B091E50170
:103A20000196A11DB11D8093E2019093E301A09343
:103A3000E401B093E501BF91AF919F918F910F90F9
:103A40000FBE0F901F9018950E94650DF8942FEFF0
:103A500087EA91E6215080409040E1F700C00000E5
:103A600087E090EBDC018093010290930202A09327
:103A70000302B09304029CE088E10FB6F894A89585
:103A8000809360000FBE90936000FFCFEF92FF9293
:103A90000F931F93CF93DF93D82FCDE08C2F0E94ED
:103AA000530405E010E0E82EF12CC701002E02C0FF
:103AB000959587950A94E2F780FF09C0602F7C2FC7
:103AC00080E00E947106D81302C081E006C0015058
:103AD000110958F7C15010F780E0DF91CF911F9185
:103AE0000F91FF90EF900895CF93C82F8CE20E9422
:103AF000461D882321F08C2FCF910C94461D80E029
:103B0000CF910895CF930E94C91E811102C00E94D7
:103B1000AF1EC5E6C15049F00E9465038FE39CE9E2
:103B20000197F1F700C00000F5CF89E20E94741DF3
:103B3000811113C18AE20E94741D81110E94AF1E7F
:103B400085E00E94741D81110E94241D0E94D41ED4
:103B50008093E00187E00E94741D8823A9F18BE126
:103B60000E94741D882351F08091E00181FB22277F
:103B700020F991E0922790FB81F90EC08EE00E941F
:103B8000741D882361F08091E00182FB222720F9D7
:103B900091E0922790FB82F98093E00115C080E1CB
:103BA0000E94741D9091E001882341F093FB22272D
:103BB00020F981E0822780FB93F904C0892F80954A
:103BC00080FB90F99093E0018091E0010E94D81E63
:103BD0000E94E61E8093000280EE0E94741D8823DE
:103BE00041F080910002982F909590FB80F980938E
:103BF000000289E30E94741D882359F0809100021D
:103C000081FB222720F991E0922790FB81F9809394
:103C1000000282EE0E94741D882359F080910002F8
:103C200082FB222720F991E0922790FB82F9809372
:103C3000000286EE0E94741D882359F080910002D4
:103C400083FB222720F991E0922790FB83F9809350
:103C5000000283EE0E94741D882359F080910002B7
:103C600084FB222720F991E0922790FB84F980932E
:103C7000000285E30E94741D882359F080910002A0
:103C800085FB222720F991E0922790FB85F980930C
:103C9000000281E30E94741D882359F08091000284
:103CA00086FB222720F991E0922790FB86F98093EA
:103CB000000281E10E94741D882359F08091000266
:103CC00087FB222720F991E0922790FB87F98093C8
:103CD0000002809100020E94EA1E8091000287FB90
:103CE000882780F980930D0187E20E94741DC82FF8
:103CF0008EE10E94741D8111C2608FE10E94741DCB
:103D00008111C46080E20E94741D8111C86081E24B
:103D10000E94741D8111C06182E20E94741D811194
:103D2000C06283E20E94741D8111C06484E20E941B
:103D3000741D882311F0C06802C0CC2329F08C2F99
:103D40000E94E11E6C2F03C00E94DD1E682F70E0F0
:103D500080E090E0CF910C94F118CF9108956DEE32
:103D60007EEF80E090E00E941B2560E082E090E022
:103D70000E94092560E083E090E00E94092560E050
:103D800084E090E00E94092560E085E090E00C94DA
:103D9000092580E090E00E94032521E08D3E9E4FA2
:103DA00009F020E0822F089582E090E00C94FB243B
:103DB000682F82E090E00C94092583E090E00C9459
:103DC000FB24682F83E090E00C94092584E090E0C8
:103DD0000C94FB24682F84E090E00C9409258091DA
:103DE000E80180FF0BC06091130185E0689FB0017E
:103DF000112475956795759567952BC081FF09C04E
:103E00006091130185E0689FB00111247595679555
:103E100020C082FF07C06091130185E0689FB00158
:103E2000112417C09091E9019923D1F060911201FA
:103E3000961788F72091130185E0289F900111249F
:103E4000929FA001939F500D112470E0CA010E941F
:103E5000CD246038710540F46115710539F002C058
:103E600065E070E0862F08958FE7089581E008955A
:103E70008091E80180FF08C06091110170E07595A4
:103E800067957595679521C081FF06C06091110106
:103E900070E07595679519C082FF04C060911101AB
:103EA00070E010C09091E9019923C1F06091100178
:103EB0009617A0F780911101899FC001112470E02D
:103EC0000E94CD246038710528F46115710521F038
:103ED000862F08958FE7089581E0089561E070E0EE
:103EE000F4CF803F21F40E94EF1E819504C0813FF2
:103EF00029F40E94EF1E8093EC010895823F21F483
:103F00000E94EF1E819504C0833F29F40E94EF1E9A
:103F10008093EB010895893F19F40E94381F05C072
:103F20008A3F31F40E94381F81958093ED010895F6
:103F30008B3F21F40E94381F819504C08C3F29F4E7
:103F40000E94381F8093EE010895843F21F48091F0
:103F5000EA01816017C0853F21F48091EA01826007
:103F600011C0863F21F48091EA0184600BC0873F35
:103F700021F48091EA01886005C0883F31F4809186
:103F8000EA0180618093EA0108958D3F21F48091D8
:103F9000E80181600BC08E3F21F48091E8018260CE
:103FA00005C08F3F29F48091E80184608093E80187
:103FB0000895803F39F48091EC0187FF6CC0109226
:103FC000EC0169C0813F29F48091EC011816BCF323
:103FD00062C09091EB01823F29F497FF5CC0109280
:103FE000EB0159C0833F19F41916CCF354C0893F33
:103FF00041F48091ED0118160CF04DC01092ED01C6
:104000004AC08A3F29F48091ED0187FF44C0F6CF72
:104010008B3F39F48091EE0187FF3DC01092EE0195
:104020003AC08C3F29F48091EE011816BCF333C0DE
:10403000843F21F48091EA018E7F17C0853F21F4EF
:104040008091EA018D7F11C0863F21F48091EA01C1
:104050008B7F0BC0873F21F48091EA01877F05C0E9
:10406000883F31F48091EA018F7E8093EA0113C08A
:104070008D3F21F48091E8018E7F0BC08E3F21F4AB
:104080008091E8018D7F05C08F3F29F48091E80180
:104090008B7F8093E8018091EB0181110EC08091AC
:1040A000EC0181110AC08091ED01811106C080915F
:1040B000EE01811102C01092E90108958AEE91E0AB
:1040C0000E947F100E94C91C9093E7018093E60133
:1040D00008951F93CF93DF938091E6019091E701BC
:1040E0000E94D51CAC019091E901992321F0209107
:1040F000140130E006C0209115018AE0289F90014C
:1041000011244217530708F486C08091EB01C09137
:10411000EC01D091ED011091EE01811107C0C111A8
:1041200076C0D11174C0111172C075C09F3F19F0D3
:104130009F5F9093E901181624F40E94EF1E80936C
:10414000EB018091EB0187FF05C00E94EF1E819576
:104150008093EB011C1624F40E94EF1E8093EC0167
:104160008091EC0187FF05C00E94EF1E819580932E
:10417000EC016091EB01662339F1C091EC01CC2395
:1041800019F1772767FD7095872F972F0E94DE23FF
:1041900023E333E343E35FE30E9442240E94AB2323
:1041A0006093EB016C2F772767FD7095872F972F12
:1041B0000E94DE2323E333E343E35FE30E944224D0
:1041C0000E94AB236093EC011D1624F40E94381F5B
:1041D0008093ED018091ED0187FF05C00E94381F9B
:1041E00081958093ED01111624F40E94381F80936D
:1041F000EE018091EE0187FF05C00E94381F819576
:104200008093EE01DF91CF911F910C945E209F3F30
:1042100009F08ECF96CFDF91CF911F910895EAEEEE
:10422000F1E085E0DF011D928A95E9F71092E9013E
:104230001092E8010895833081F128F4813059F01B
:104240008230D1F00895853009F449C0B8F1863044
:1042500009F456C0089580911501262F30E0280FEB
:10426000311D2F3F310524F4680F60931501089527
:104270008FEF80931501089580911401262F30E06F
:10428000280F311D2F3F310524F4680F609314016E
:1042900008958FEF80931401089580911301262FC4
:1042A00030E0280F311D2F3F310524F4680F609353
:1042B000130108958FEF80931301089580911201E7
:1042C000262F30E0280F311D2F3F310524F4680FD1
:1042D0006093120108958FEF8093120108958091E9
:1042E0001101262F30E0280F311D2F3F310524F416
:1042F000680F6093110108958FEF80931101089565
:1043000080911001262F30E0280F311D2F3F3105FD
:1043100024F4680F6093100108958FEF80931001CB
:104320000895833011F128F4813049F0823091F002
:104330000895853081F120F18630C1F10895809192
:104340001501681720F4861B8093150108951092BB
:104350001501089580911401681720F4861B80933D
:1043600014010895109214010895809113016817A3
:1043700020F4861B80931301089510921301089571
:1043800080911201681720F4861B80931201089512
:1043900010921201089580911101681720F4861B74
:1043A00080931101089510921101089580911001D8
:1043B000681720F4861B8093100108951092100155
:1043C00008950F931F938D3109F46BC008F03FC01F
:1043D0008E3009F47FC0C0F4873009F469C068F4F6
:1043E000863009F0B1C08091E001817F8E7F80939B
:1043F000E00181E08093F001A8C0883009F4A2C0F8
:104400008B3009F49FC0A0C0863109F49BC078F4BA
:10441000803109F472C0813109F096C00E943115D3
:1044200090910D0181E0892780930D018BC0893126
:1044300009F488C08B3109F087C08091E00181FBCD
:10444000222720F991E0922790FB81F94CC0853317
:1044500009F470C048F4873209F46CC008F459C0FC
:10446000893209F467C070C0833438F48A3308F0A5
:104470004EC0883309F466C067C0833409F45AC05B
:10448000883409F061C00E9431150FEF13ED20E36D
:10449000015010402040E1F700C000000E94241DA0
:1044A00051C00E9465230E9468100E9461094AC0A1
:1044B0009091E001892F8095817080FB90F929F01F
:1044C000966098609093E00140C0997F977F9093A9
:1044D000E00138C08091E00182FB222720F991E0C1
:1044E000922790FB82F98093E001992359F1809102
:1044F000E00181608093E00125C08091E00183FBB1
:10450000222720F991E0922790FB83F9ECCF895381
:1045100001C08D5141E050E060E070E08A019B01F4
:1045200004C0000F111F221F331F8A95D2F7C90143
:10453000B80104C061E070E080E090E00E94F118F2
:104540000E94311581E001C080E01F910F91089514
:1045500080E0089580E00895CF93C82F8091F00106
:10456000813079F018F08230E9F187C0E0910E01D6
:10457000F0910F018081813169F0823209F07FC0B2
:1045800009C0E0910E01F0910F018081813111F09D
:10459000823261F48C2F0E94A822811104C08C2FDA
:1045A0000E94E1211DC081E090E01AC08C2F0E9482
:1045B000AA22811114C0C43179F048F4CB3079F0CB
:1045C000C03109F060C082E08093F00108C0C932B8
:1045D00019F0C83321F057C01092F00154C081E0A7
:1045E000817053C0C93289F118F5C43171F1A8F452
:1045F000C73009F046C08AE08093150194E190939A
:10460000140193E0909313018093120188E080934A
:10461000110188E28093100134C0CE51C63088F574
:10462000EC2FF0E0E65DFE4F80818093EF0129C022
:10463000CE34E9F020F4CB3421F56AE013C0C13563
:1046400079F0C235F1F461E00DC08091EF0188236B
:1046500019F01092EF0115C081E08093F00115C0B0
:1046600061E006C08091EF010E941B210AC06AE050
:104670008091EF010E94912104C01092F00180E02E
:1046800004C081E002C080E0ABCFCF910895E1E8A3
:10469000F0E08081886080838081816080838FB733
:1046A000F89493E09093890090ED909388008FBFE9
:1046B0000895EFE6F0E08081826080830895EFE660
:1046C000F0E080818D7F80830895EFE6F0E09081B7
:1046D00082E08927808308951F920F920FB60F9270
:1046E00011242F933F934F935F936F937F938F93F7
:1046F0009F93AF93BF93EF93FF938091F1019091BC
:10470000F20101969093F2018093F101811103C0AF
:1047100082E00E946109E091F201E695E695F0E001
:10472000E851FB4FE4918091F1018E1303C080E0CA
:104730000E946109FF91EF91BF91AF919F918F917D
:104740007F916F915F914F913F912F910F900FBE8D
:104750000F901F90189504D06894B1118DC00895E2
:1047600070D088F09F5790F0B92F9927B751A0F0DB
:10477000D1F0660F771F881F991F1AF0BA95C9F7F5
:1047800012C0B13081F077D0B1E0089574C0672FC6
:10479000782F8827B85F39F0B93FCCF386957795A5
:1047A0006795B395D9F73EF490958095709561958E
:1047B0007F4F8F4F9F4F0895E89409C097FB3EF4B9
:1047C00090958095709561957F4F8F4F9F4F99235E
:1047D000A9F0F92F96E9BB279395F69587957795DC
:1047E0006795B795F111F8CFFAF4BB0F11F460FF9C
:1047F0001BC06F5F7F4F8F4F9F4F16C0882311F0F4
:1048000096E911C0772321F09EE8872F762F05C007
:10481000662371F096E8862F70E060E02AF09A95A2
:10482000660F771F881FDAF7880F9695879597F997
:10483000089557FD9058440F551F59F05F3F71F090
:104840004795880F97FB991F61F09F3F79F08795F7
:104850000895121613061406551FF2CF4695F1DF80
:1048600008C0161617061806991FF1CF8695710510
:10487000610508940895E894BB2766277727CB0144
:1048800097F908950BD078C069D028F06ED018F051
:10489000952309F05AC05FC01124EECFCADFA0F300
:1048A000959FD1F3950F50E0551F629FF001729FC5
:1048B000BB27F00DB11D639FAA27F00DB11DAA1FE4
:1048C000649F6627B00DA11D661F829F2227B00D31
:1048D000A11D621F739FB00DA11D621F839FA00DBC
:1048E000611D221F749F3327A00D611D231F849F0C
:1048F000600D211D822F762F6A2F11249F57504063
:104900008AF0E1F088234AF0EE0FFF1FBB1F661FFD
:10491000771F881F91505040A9F79E3F510570F0B6
:1049200014C0AACF5F3FECF3983EDCF386957795F1
:104930006795B795F795E7959F5FC1F7FE2B880FB1
:10494000911D9695879597F9089597F99F6780E847
:1049500070E060E008959FEF80EC089500240A94D1
:104960001616170618060906089500240A9412164A
:104970001306140605060895092E0394000C11F47D
:10498000882352F0BB0F40F4BF2B11F460FF04C02A
:104990006F5F7F4F8F4F9F4F089597FB072E16F441
:1049A000009407D077FD09D00E94E72407FC05D0CA
:1049B0003EF4909581959F4F0895709561957F4F36
:1049C0000895EE0FFF1F0590F491E02D0994AA1BA6
:1049D000BB1B51E107C0AA1FBB1FA617B70710F0EA
:1049E000A61BB70B881F991F5A95A9F7809590951C
:1049F000BC01CD010895F999FECF92BD81BDF89A11
:104A0000992780B50895A8E1B0E042E050E00C9409
:104A10002325262FF999FECF92BD81BDF89A0197E3
:104A200000B4021639F01FBA20BD0FB6F894FA9AF6
:104A3000F99A0FBE08950196272F0E940A250C941B
:104A40000925DC01CB01FC01F999FECF06C0F2BDBE
:104A5000E1BDF89A319600B40D9241505040B8F73C
:064A60000895F894FFCF59
:104A660002206309F109CE099A0966090101CD01FF
:104A760028080A03140A3F4D3639A9045C042604A3
:104A8600ED0380039903B203CB0301020304050679
:044A96000708090004
:00000001FF
